:100000000C94FE070C9426080C9426080C942608E1
:100010000C9426080C9426080C9426080C942608A8
:100020000C9426080C9426080C943D0E0C94430F57
:100030000C9426080C9426080C9426080C94260888
:100040000C9426080C94B80A0C9426080C942608E4
:100050000C9426080C9426080C9426080C946E0A1E
:100060000C9426080C9426080C9426080C94260858
:100070000C9426080C9426080C9426080C94260848
:100080000C94C30B0C9426080C9426080C94260898
:100090000C9426080C9426080C9426080C94260828
:1000A0000C9426080C9426080C942608F0F89C8ED4
:1000B0008783878E9CF8F00000FEFF030303030391
:1000C000070EFCF80000FEFF0303030303070EFC0A
:1000D000F80000FFFF00000000000000FFFF00002C
:1000E000FEFF8383838383C7EE7C380000F8FC0E19
:1000F00007030303070EFCF800003F7FE0C0808089
:10010000C0E07F3FFFFF01010101010101FFFF008E
:1001100000FFFF0C0C0C0C1C3E77E3C100007FFFBE
:10012000C0C0C0C0C0E0703F1F00001F3F70E0C0F3
:10013000C0C0E0703F1F00007FFFC1C1C1C1C1E36B
:10014000773E1C00001F3F70E0C0C0C0E0703F1F42
:10015000000000000001FFFF01000000D5F08D1439
:10016000A1C881CFD9F1AF2000070605040100081E
:100170000A0B0C0D099028039B904301CD90400180
:10018000CD9045913C922A039B9042913982039BEA
:10019000902B81039B90479137039B904391399219
:1001A0002D039B904291398201CD9045913601CD2E
:1001B000902F81039B904301CD904001CD904C91B5
:1001C000360736924001CD9030818201CD902C03CC
:1001D0009B904A913E039B903E912D039B904891AA
:1001E0003C039B90479143923B9328039B90439100
:1001F00028828301CD90408101CD90439139923086
:10020000039B9042913B922F039B9040913B9237EE
:100210009328039B818283073691280930912A090C
:1002200030912B0930912D09309134922809309169
:1002300034922A09309134922B09309134922D094D
:100240003091349228024C90408182024C904C02B2
:100250004C9040024C9034912A0498904C81024C6E
:100260009040024C9034912B024C904081024C9073
:100270004C024C9040024C9034912D0498904C814B
:10028000024C9040024C9043913B92349328024C94
:1002900090408182024C904C024C9040024C904322
:1002A000913B9234932A0498904C818283024C9023
:1002B000400126904201269043913B9234932B02B9
:1002C0004C9040818283024C904C024C904001261D
:1002D0009042012690459134922D0498904C818251
:1002E000024C9040024C9043913B92349328024C34
:1002F00090408182024C904C024C9040024C9043C2
:10030000913B9234932A0498904C818283024C90C2
:10031000400126904201269043913B9234932B0258
:100320004C9040818283024C904C024C90400126BC
:100330009042012690459134922D0498904C8182F0
:10034000024C9040024C9040913B9228024C9040CD
:10035000913B024C9040913B024C9040913B024CAF
:1003600090409139922A024C90409139024C904031
:100370009139024C90409139024C903B9137922B2D
:10038000024C903B9137024C903B9137024C903B92
:100390009137024C903B9139922D024C903B913910
:1003A000024C903B9139024C903B9139024C904069
:1003B000913B9228024C9040913B024C9040913BE3
:1003C000024C9040913B024C90409139922A024C51
:1003D00090409139024C90409139024C90409139B3
:1003E000024C903B9137922B024C903B9137024C40
:1003F000903B9137024C903B9137024C903B9139A6
:10040000922D024C903B9139024C903B9139024C19
:10041000903B9139024C9040913B92280126903BB1
:100420008101269040913B0126903B81012690431B
:100430009140933B024C90429140933B0126904067
:100440008183012690409139922A0126903B8101B7
:1004500026904091390126903B810126904391409E
:100460009339024C90429140933901269040818308
:100470000126903B9137922B0126903B81012690DB
:1004800040913B93370126903B8183012690439115
:100490003B9337024C9042913B9337012690408129
:1004A000830126903B9139922D0126903B810126B4
:1004B0009040913B93390126903B818301269043E4
:1004C000913B9339024C9042913B933901269040E5
:1004D000818301269040913B92280126903B810127
:1004E000269040913B0126903B810126904391400C
:1004F000933B024C90429140933B01269040818374
:10050000012690409139922A0126903B8101269044
:100510004091390126903B810126904391409339C7
:10052000024C9042914093390126904081830126EC
:10053000903B9137922B0126903B81012690409170
:100540003B93370126903B818301269043913B9357
:1005500037024C9042913B933701269040818301B2
:1005600026903B9139922D0126903B8101269040A7
:10057000913B93390126903B818301269043913B27
:100580009339024C9042913B9339012690408183EC
:100590000126902882029A9140014D913B014D9194
:1005A00043014D913B014D9140014D913B014D90D7
:1005B00045912A014D903B014D903F014D903B01EB
:1005C0004D9042014D903B014D903F014D903B01BC
:1005D0004D902B81014D913B014D9140014D913B3F
:1005E000014D904781014D903B014D9043014D904D
:1005F0003B014D9043912D014D9039014D903C01AF
:100600004D9039014D9042014D903C014D90450176
:100610004D903C014D902F81014D913B014D9140FA
:10062000014D913B014D904381014D9040014D9012
:1006300047014D9043014D904C9130014D90400148
:100640004D9043014D9040014D9048014D90430124
:100650004D904C014D9043014D904C912C014D908B
:100660004081014D9044014D9040014D9047014D16
:100670009044014D904A014D9044014D904A912D76
:10068000014D9040014D9045014D904A014D9048DB
:100690009245014D904082014D9045014D90480199
:1006A0004D90479128014D903B014D9040014D9058
:1006B0003B014D9043014D903B014D9040014D90C9
:1006C0003B014D9043912D014D9039014D903C01DE
:1006D0004D9043014D9042912F014D9039014D9025
:1006E0003B014D903F014D90409128014D903B01C1
:1006F0004D9043014D903B014D9040014D903B0189
:100700004D9043014D9040014D904781014D9043E4
:10071000014D904C014D9047014D904F014D904C33
:10072000014D9053014D904F014D9028029A9140F8
:10073000014D913B014D9143014D913B014D914044
:10074000014D913B014D9045912A014D903B014D4A
:10075000903F014D903B014D9042014D903B014D2A
:10076000903F014D903B014D902B81014D913B01FC
:100770004D9140014D913B014D904781014D903B82
:10078000014D9043014D903B014D9043912D014D02
:100790009039014D903C014D9039014D9042014DF1
:1007A000903C014D9045014D903C014D902F8101B1
:1007B0004D913B014D9140014D913B014D90438145
:1007C000014D9040014D9047014D9043014D904C9B
:1007D0009130014D9040014D9043014D9040014DAD
:1007E0009048014D9043014D904C014D9043014D77
:1007F000904C912C014D904081014D9044014D90C1
:1008000040014D9047014D9044014D904A014D905B
:1008100044014D904A912D014D9040014D9045016C
:100820004D904A014D90489245014D904082014DB6
:100830009045014D9048014D90479128014D903BC6
:10084000014D9040014D903B014D9043014D903B37
:10085000014D9040014D903B014D9043912D014D34
:100860009039014D903C014D9043014D9042912FA4
:10087000014D9039014D903B014D903F014D90400D
:100880009128014D903B014D9043014D903B014D0E
:100890009040014D903B014D9043014D9040014DE2
:1008A000904781014D9043014D904C014D9047017F
:1008B0004D904F014D904C014D9053014D904F0183
:1008C0004D90280A6A902A0535904A01F390480114
:1008D000F3904700A6904500A69047912B00A69064
:1008E0004800A6904700A6904500A69047029A812E
:1008F0000535902D0535914501F39143014D914208
:1009000000A6914000A6914200A69043912F00A618
:10091000904200A6904000A6904203418005359089
:10092000308107CF9040014D9040006F903E006FA6
:10093000903C006F903B912C0A6A902D81091D908C
:100940003C006F903B006F9039006F903691280A01
:100950006A902D810A6A90280A6A80F001020408D0
:100960001020408000000000003E5B4F5B3E3E6B6D
:100970004F6B3E1C3E7C3E1C183C7E3C181C577D39
:10098000571C1C5E7F5E1C00183C1800FFE7C3E785
:10099000FF0018241800FFE7DBE7FF30483A060E97
:1009A0002629792926407F050507407F05253F5ADE
:1009B0003CE73C5A7F3E1C1C08081C1C3E7F14224E
:1009C0007F22145F5F005F5F06097F017F006689F9
:1009D000956A606060606094A2FFA29408047E043F
:1009E0000810207E201008082A1C08081C2A080865
:1009F0001E101010100C1E0C1E0C30383E38300625
:100A00000E3E0E06000000000000005F0000000720
:100A1000000700147F147F14242A7F2A122313084E
:100A2000646236495620500008070300001C22412A
:100A3000000041221C002A1C7F1C2A08083E0808CE
:100A4000008070300008080808080000606000207E
:100A5000100804023E5149453E00427F4000724961
:100A60004949462141494D331814127F1027454505
:100A700045393C4A4949314121110907364949491B
:100A800036464949291E0000140000004034000089
:100A900000081422411414141414004122140802F2
:100AA000015909063E415D594E7C1211127C7F4965
:100AB0004949363E414141227F4141413E7F4949BA
:100AC00049417F090909013E414151737F080808E6
:100AD0007F00417F41002040413F017F08142241B7
:100AE0007F404040407F021C027F7F0408107F3E11
:100AF0004141413E7F090909063E4151215E7F097E
:100B0000192946264949493203017F01033F4040E4
:100B1000403F1F2040201F3F4038403F63140814CF
:100B20006303047804036159494D43007F41414107
:100B30000204081020004141417F040201020440E8
:100B400040404040000307080020545478407F286C
:100B50004444383844444428384444287F38545462
:100B6000541800087E090218A4A49C787F08040485
:100B70007800447D40002040403D007F1028440024
:100B800000417F40007C047804787C0804047838B5
:100B900044444438FC1824241818242418FC7C08E5
:100BA000040408485454542404043F44243C404062
:100BB000207C1C2040201C3C4030403C4428102815
:100BC000444C9090907C4464544C4400083641005E
:100BD0000000770000004136080002010204023CD8
:100BE0002623263C1EA1A161123A4040207A3854A7
:100BF0005455592155557941215454784121555422
:100C0000784020545579400C1E5272123955555572
:100C100059395454545939555454580000457C415D
:100C20000002457D420001457C40F0292429F0F076
:100C3000282528F07C545545002054547C547C0AC7
:100C4000097F4932494949323248484832324A4894
:100C500048303A4141217A3A42402078009DA0A094
:100C60007D39444444393D4040403D3C24FF2424E8
:100C7000487E4943662B2FFC2F2BFF0929F620C005
:100C8000887E090320545479410000447D41304856
:100C9000484A32384040227A007A0A0A727D0D1999
:100CA000317D2629292F28262929292630484D40FB
:100CB00020380808080808080808382F10C8ACBAF7
:100CC0002F102834FA00007B000008142A14222276
:100CD000142A14089500220095AA005500AAAA55C6
:100CE000AA55AA000000FF00101010FF00141414F1
:100CF000FF001010FF00FF1010F010F0141414FC8F
:100D0000001414F700FF0000FF00FF1414F404FCAB
:100D1000141417101F10101F101F1414141F00108C
:100D20001010F0000000001F101010101F10101005
:100D300010F010000000FF10101010101010101014
:100D4000FF10000000FF140000FF00FF00001F1054
:100D5000170000FC04F414141710171414F404F40E
:100D60000000FF00F714141414141414F700F714FF
:100D70001414171410101F101F141414F41410104E
:100D8000F010F000001F101F0000001F14000000F2
:100D9000FC140000F010F01010FF10FF141414FFEA
:100DA000141010101F00000000F010FFFFFFFFFFE5
:100DB000F0F0F0F0F0FFFFFF0000000000FFFF0F79
:100DC0000F0F0F0F38444438447C2A2A3E147E0209
:100DD000020606027E027E0263554941633844449E
:100DE0003C04407E201E2006027E020299A5E7A553
:100DF000991C2A492A1C4C7201724C304A4D4D30C4
:100E00003048784830BC625A463D3E494949007EE8
:100E10000101017E2A2A2A2A2A44445F444440517F
:100E20004A444040444A51400000FF0103E080FF33
:100E3000000008086B6B083612362436060F090FBF
:100E400006000018180000001010003040FF0101DB
:100E5000001F01011E00191D1712003C3C3C3C0004
:100E60000000000000000000240027002A002D00E0
:100E7000300000000000250028002B002E0031006B
:100E80000408020110408040102040804080080289
:100E900004018040201002011080102040402004F6
:100EA0000404040403040502020202040302020211
:100EB00002060606060606040402020204040601EF
:100EC0001501260137014A015D01720188019F0168
:100ED000B801D201EE010B022A024B026E0293020C
:100EE000BA02E40210033F037003A403DC031704F7
:100EF00055049704DD0427057505C80520067D0601
:100F0000E0064907B8072D08A9082D09B9094D0AB7
:100F1000EA0A900B400CFA0CC00D910E6F0F5A109C
:100F200053115B1272139A14D41520178018F519F7
:100F3000801B231DDE1EB420A622B524E4263429FE
:100F4000A72B402E0031EA330037453ABC3D6841BB
:100F50004C456B49C84D68524F57805C0062101178
:100F60001213151617181A1C1D1F21232527292CAB
:100F70002E3134373A3E4145494E52575C62686ED5
:100F8000757B838B939CA5AFB9C4D0DCE9F7080BC4
:100F90000002020201000904000001020200000533
:100FA0002400100105240101010424020605240681
:100FB00000010705810310004009040100020A0036
:100FC0000000070502024000000705830240000000
:100FD0000403090412010002EF020140412336809C
:100FE00000010102030141726475696E6F204C4C6F
:100FF000430041726475626F7900361511241FBE7B
:10100000CFEFDAE0DEBFCDBF11E0A0E0B1E0E0E776
:10101000FDE202C005900D92AA33B107D9F726E090
:10102000AAE3B1E001C01D92A938B207E1F717E0C9
:10103000CEEFD7E004C02197FE010E94AB16CD3F52
:10104000D107C9F70E9473110C94B6160C940000D6
:10105000CF92DF92EF92FF920F931F93CF93DF9384
:101060006C017A018B01C0E0D0E0CE15DF0589F07C
:10107000D8016D918D01D601ED91FC910190F08127
:10108000E02DC6010995892B11F47E0102C021963D
:10109000ECCFC701DF91CF911F910F91FF90EF909F
:1010A000DF90CF9008953FB7F8948091FE01909122
:1010B000FF01A0910002B091010226B5A89B05C0D6
:1010C0002F3F19F00196A11DB11D3FBFBA2FA92FC7
:1010D000982F8827820F911DA11DB11DBC01CD0144
:1010E00042E0660F771F881F991F4A95D1F7089530
:1010F000CF92DF92EF92FF921F93CF93DF93E82F6F
:10110000F0E0E05FFE4F1081E62FF0E0603330F456
:10111000E25AF04FE491CE2FD0E006C0EE0FFF1F51
:10112000E25AF14FC591D4916E01E12CF12C60E0AF
:1011300074E284EF90E0A70196010E942016DA0184
:10114000C9010197A109B109009721E0A207B105E2
:1011500078F060E970ED83E090E0A70196010E94CD
:101160002016DA01C9010197A109B10923E001C0E4
:1011700021E01130C9F0133051F530919100387FE2
:10118000232B209391009093990080939800D09303
:10119000FB01C093FA0181E08093F9018091710015
:1011A00082608093710013C03091FC0131110FC037
:1011B00030918100387F232B209381009093890008
:1011C0008093880080916F00826080936F00DF9130
:1011D000CF911F91FF90EF90DF90CF900895E82F6F
:1011E000F0E0E05FFE4F8081813019F0833089F0BC
:1011F00008958091FC01811122C080916F008D7F44
:1012000080936F009091EB01E091E901F091EA0188
:101210000CC01092F9018091F801811110C09091D9
:10122000F601E091F401F091F5018081282F30E082
:10123000892F90E080959095822393238083089551
:101240008091E40108952F923F924F925F926F92A6
:101250007F928F929F92AF92BF92CF92DF92EF9246
:10126000FF920F931F93CF93DF93CDB7DEB72797EE
:101270000FB6F894DEBF0FBECDBF9B838A836A3062
:10128000A1F4DC015C962C915C9758968D919C9111
:101290005997B8E02B9F800D911D1124EA81FB81A5
:1012A000918F808F178A168AC1C06D3009F4BEC035
:1012B000AA81BB815C964C915C975B966C905B9726
:1012C0006E825A967C905A977F825896CD90DC9089
:1012D000599756968D919C91579780389105C4F0F7
:1012E000AA81BB815C962C915C97422F50E0569668
:1012F0008D919C915797B6E02B9F800D911D1124E5
:10130000EA81FB81978B868B258D21117AC08EC057
:10131000F0E4CF16D10424F79C0155E0459F200D41
:10132000311D112412161306DCF6242E312C9601E1
:10133000A8E04A9F200D311D11241216130684F6D1
:10134000B5E06B9FB0011124FB01EC59F64F2F0162
:1013500050E0F201B490553009F4B12C7601B8E0B8
:101360009B2EB0FC02C08E8001C08F8081100BC00C
:101370006E807F80671007C0B6949A94E20CF31CCD
:101380009110EFCF33C09C012983622F681B641733
:1013900098F7B701E62FEE19E41728F52038310544
:1013A000F8F460347105E0F48B01ECE5F9E0A0E1BC
:1013B0006A2E7980609ED001A0781124A70D077055
:1013C000E00FF11DA490BD83AC83AB5FBD4F8820BF
:1013D00019F0EC91AE2A03C0A094EC91AE22AC922D
:1013E0006F5F7F4FD7CF2F5F3F4FCECF5F5F820DB5
:1013F000931D92012F5F3F4F2901563009F0A9CF6D
:101400006FCF6AEF64039001659F300D112420585F
:101410003F4F2817390754F48A819B81DC01ED91F5
:10142000FC910190F081E02D6AE0099581E090E067
:1014300027960FB6F894DEBF0FBECDBFDF91CF91D8
:101440001F910F91FF90EF90DF90CF90BF90AF90E2
:101450009F908F907F906F905F904F903F902F90D4
:10146000089508950E94B1168F929F92AF92BF92F5
:10147000CF92DF92EF92FF926B017C010E945308A2
:101480004B015C01C114D104E104F104F1F00E94AC
:101490005308DC01CB0188199909AA09BB09883EC8
:1014A0009340A105B10570F321E0C21AD108E1080B
:1014B000F10888EE880E83E0981EA11CB11CC114AF
:1014C000D104E104F10419F7DDCFFF90EF90DF9034
:1014D000CF90BF90AF909F908F9008951F920F92E2
:1014E0000FB60F9211242F933F938F939F93AF9337
:1014F000BF9380913F0190914001A0914101B09133
:1015000042013091FD0123E0230F2D3720F4019695
:10151000A11DB11D05C026E8230F0296A11DB11D16
:101520002093FD0180933F0190934001A0934101DE
:10153000B09342018091FE019091FF01A0910002C1
:10154000B09101020196A11DB11D8093FE019093FF
:10155000FF01A0930002B0930102BF91AF919F9150
:101560008F913F912F910F900FBE0F901F90189564
:101570001F920F920FB60F9211242F933F938F93C8
:101580009F93AF93BF93EF93FF938091FC018823C8
:1015900009F44FC08091EC019091ED01A091EE0112
:1015A000B091EF01892B8A2B8B2B51F18091EB01AC
:1015B000E091E901F091EA0190818927808380918F
:1015C000EC019091ED01A091EE01B091EF011816A0
:1015D00019061A061B06D4F58091EC019091ED01D5
:1015E000A091EE01B091EF010197A109B10980939B
:1015F000EC019093ED01A093EE01B093EF0126C0B2
:101600001092F8011092FC0180916F008D7F809301
:101610006F009091EB01E091E901F091EA01808186
:10162000282F30E0892F90E0809590958223932396
:101630000CC08091F701811109C08091EB01E0910C
:10164000E901F091EA01908189278083FF91EF9170
:10165000BF91AF919F918F913F912F910F900FBEAE
:101660000F901F901895CF93DF93D1E0E0913A014E
:10167000F0913B019F012F5F3F4F30933B0120933F
:101680003A018491982F907FC82FCF70903821F421
:101690008C2F0E94EF08EACF9039F9F4E09105060B
:1016A000F091060609958D278093F701E0913A01A4
:1016B000F0913B01CF01019690933B0180933A0159
:1016C00064918091E801C81788F6C13009F052C0D2
:1016D0008091E7018111CACF4DC097FD3AC0329683
:1016E000F0933B01E0933A01F901249130E0382B6B
:1016F000A091FA01B091FB010E9474166C507E4FCC
:101700008F4F9F4F28EE33E040E050E00E9452168A
:101710002093F0013093F1014093F2015093F301D3
:101720008091F0019091F101A091F201B091F3014B
:10173000892B8A2B8B2B21F581E090E0A0E0B0E093
:101740008093F0019093F101A093F201B093F30123
:1017500017C0903E49F480913C0190913D019093D7
:101760003B0180933A0182CF903F09F07FCF1092E6
:101770003E0106C067FD7ACF8C2F0E94780876CF95
:10178000DF91CF9108951F920F920FB60F921124FF
:101790002F933F934F935F936F937F938F939F9379
:1017A000AF93BF93EF93FF938091F901882341F0AA
:1017B0008091F801811104C08091F701882351F1D3
:1017C00080913E01882381F18091F0019091F10197
:1017D000A091F201B091F301892B8A2B8B2B21F17F
:1017E0008091F0019091F101A091F201B091F3018B
:1017F0000197A109B1098093F0019093F101A093A1
:10180000F201B093F301892B8A2B8B2B69F40E9490
:10181000330B0AC08091F601E091F401F091F501DB
:10182000908189278083CCCFFF91EF91BF91AF91B9
:101830009F918F917F916F915F914F913F912F91E8
:101840000F900FBE0F901F9018959091E801923065
:1018500009F471C0292F30E0F901E05FFE4F4081AB
:10186000F901EB51FE4F8083913031F42091E50175
:10187000281302C09093E7019F5F9093E80190E0E6
:10188000FC01E156F14F2491FC01E058F14F8491A5
:1018900030E0220F331FF901EE58F14F659174913A
:1018A000F901EC59F14FA591B4919C91982B9C931F
:1018B000413019F04330D9F0089590916400977F3A
:1018C00090936400109280001092810090918100AA
:1018D0009860909381009091810091609093810035
:1018E0007093EA016093E9018093EB010895909170
:1018F0006500977F90936500109290001092910080
:1019000090919100986090939100909191009160D6
:10191000909391007093F5016093F4018093F60128
:101920008091E801882321F06CE380E00E94780830
:1019300080E00C94EF0808952D9A0895BC0180E092
:1019400090E00C94340A8FB18095807F669B88600C
:101950001C9B8460089583B7817F83BF83B78160B8
:1019600083BF889583B78E7F83BF08958EBD0000A7
:101970000DB407FEFDCF08955C980E94B60C5C9AEA
:1019800008951092E4013E983F9808953E9A3F9A38
:1019900081E08093E4010895FC01809104028111AB
:1019A00003C08FEF9FEF08959FB7F89482E0809374
:1019B000E9002091F20030E01216130614F421E041
:1019C00030E02115310559F0289884E68093030210
:1019D0008091F10080838091F200882319F09FBFED
:1019E000C90108958BE68093E800F9CFCF93DF9388
:1019F0001F92CDB7DEB76983DC01ED91FC910280C7
:101A0000F381E02D41E050E0BE016F5F7F4F09950B
:101A10000F90DF91CF91089583E08093E90080914A
:101A2000F200882319F08AE38093E8000895CF93A9
:101A3000DF931F92CDB7DEB7FC018485958597FDB6
:101A400005C02FEF3FEF358724870BC0CE010196ED
:101A50000E94CC0C019719F4898190E002C08FEFAD
:101A60009FEF0F90DF91CF9108950F931F93CF9326
:101A7000DF931F92CDB7DEB78C01FC01848595857D
:101A800097FF0EC0CE0101960E94CC0C019719F46D
:101A9000298130E002C02FEF3FEFF801358724871E
:101AA000F801848595850F90DF91CF911F910F915B
:101AB0000895FC018485958597FD0BC09FB7F89428
:101AC00082E08093E9008091F2009FBF90E0019650
:101AD00008959FB7F89482E08093E9008091F20026
:101AE0009FBF90E008957F928F929F92AF92BF9296
:101AF000CF92DF92EF92FF920F931F93CF93DF93DA
:101B00006C015B017A0180910701882309F46BC0A5
:101B100080910402882309F466C08091020280FF4C
:101B200005C08091E00082608093E000E70110E052
:101B30000AEF83E0982E90E4792E2AE3822E2097F4
:101B400009F448C08FB7F8949092E9009091E800AA
:101B500095FF06C09091F200272D291B922F01C0FE
:101B600090E08FBF91110AC0015009F43CC061E0C0
:101B700070E080E090E00E94340AE1CF292F30E04D
:101B8000C217D3070CF49C2F8FB7F8949092E900FA
:101B90002091E80025FF1CC0292F30E0C21BD30B89
:101BA000F501915020F041914093F100FACFA20E3F
:101BB000B31E112319F08092E80009C09091E8004B
:101BC00095FD06C08092E80011E0209709F010E032
:101BD0008FBFB5CF1111B6CF5D9884E680932606EE
:101BE0001E141F0444F081E090E0F6019383828389
:101BF00080E090E001C0C701DF91CF911F910F916C
:101C0000FF90EF90DF90CF90BF90AF909F908F901C
:101C10007F90089580E0E5E0F2E081118FEF0024ED
:101C200081938193819381930394D1F70895809157
:101C300005028EBDE6E0F2E081910DB407FEFDCF16
:101C40008EBD86E0E530F807B9F70DB407FEFDCF8D
:101C5000089580912B0681110DC082E080932706A4
:101C600084E08093280610922A061092290681E0CB
:101C700080932B0687E296E008951F920F920FB68D
:101C80000F9211248F939F938091E1009091E10036
:101C9000937F9093E10083FF0FC01092E90091E0E1
:101CA0009093EB001092EC0092E39093ED00109271
:101CB000040298E09093F00082FF20C093E090939C
:101CC000E9009091F200992319F09AE39093E800CB
:101CD00090912606992339F0909126069150909381
:101CE0002606992389F190910302992339F0909166
:101CF0000302915090930302992341F184FF10C095
:101D00008091E2008E7E81608093E2008091E1000C
:101D10008F7E8093E100809102028E7E806111C0EF
:101D200080FF16C08091E2008E7E80618093E20089
:101D30008091E1008E7E8093E100809102028E7E90
:101D400081608093020204C05D9ACDCF289AD6CFDD
:101D50009F918F910F900FBE0F901F9018954091FB
:101D60008706509188062091850630918606421795
:101D70005307B4F49091E8009570E1F39091E80076
:101D800092FD19C08093F10080918706909188069A
:101D900001968F739927892B19F48EEF8093E800B1
:101DA000809187069091880601969093880680938B
:101DB000870681E0089580E00895DF92EF92FF9218
:101DC0000F931F93CF93DF93D82E8A017B01E40EEC
:101DD000F51EEB01CE15DF0571F0D7FE03C0FE0145
:101DE000849101C088810E94AF0E21968111F2CFAB
:101DF0008FEF9FEF01C0C801DF91CF911F910F912D
:101E0000FF90EF90DF900895615030F02091F10045
:101E1000FC0120830196F8CF289884E68093030282
:101E200008950F931F93CF93DF931F92CDB7DEB723
:101E300082E0898342E450E06EE87FE080E80E941F
:101E4000DD0E0E94290EDC0112960D911C91139754
:101E50000115110569F0D801ED91FC910280F38123
:101E6000E02DBE016F5F7F4FC801099597FF07C046
:101E700089810F90DF91CF911F910F910895F80103
:101E800000851185E5CF1F920F920FB60F92112496
:101E9000CF92DF92EF92FF920F931F932F933F9376
:101EA0004F935F936F937F938F939F93AF93BF9362
:101EB000EF93FF93CF93DF93CDB7DEB76C97DEBF81
:101EC000CDBF1092E9008091E80083FFEDC168E08A
:101ED000CE0145960E94040F82EF8093E8008D8921
:101EE00087FF05C09091E80090FFFCCF03C09EEFF4
:101EF0009093E800982F907609F0C6C09E892F89AC
:101F0000188D91110CC0803829F48091840680933B
:101F1000F10002C01092F1001092F10048C1422F6E
:101F200050E0512B913051F4811141C141305105A4
:101F300009F03DC1809184068D7F0BC0933061F420
:101F4000811135C14130510509F031C180918406BC
:101F50008260809384062BC1953041F48091E80023
:101F600080FFFCCF20682093E30021C1963009F068
:101F70005FC0EB8CFC8C1092E900109288061092E6
:101F80008706123091F510928606109285060E94FF
:101F9000110F99E0BE016F5F7F4FDB01E92F1D92AA
:101FA000EA95E9F799831A8391E09E8390EA9887EE
:101FB0009AEF99872091870630918806275F3F4FD7
:101FC0003C832B838D831092E90010928806109237
:101FD0008706F0928606E092850649E050E080E0B0
:101FE0000E94DD0E0E94110FE2C0F0928606E09280
:101FF00085060E94290EDC011296ED90FC90139745
:10200000E114F10409F4C0C0D701ED91FC91048002
:10201000F581E02DBE016B5E7F4FC70109950097EA
:1020200019F00CF0C4C0C7C0F701E084F184E8CF18
:10203000973009F4C0C0983021F481E08093F1001A
:10204000B6C0993009F0B3C0837009F0B4C0E3E3BF
:10205000F1E081E021E036E39081992361F0809303
:10206000E9002093EB0091919093EC003093ED0008
:102070008F5F873089F78EE78093EA001092EA003D
:102080008F898093040293C08B8D9C8D1092E90000
:102090001092880610928706909386068093850694
:1020A000898D811156C08E899D89913A59F481326A
:1020B00009F081C047E050E060E071E080E00E94FC
:1020C000DD0E75C0913209F076C0833289F4888DB7
:1020D00090E0982F88272F89822BA0E0B0E0809392
:1020E000080190930901A0930A01B0930B015FC00E
:1020F000803269F48091E80082FFFCCF67E080E0E5
:1021000091E00E94040F8BEF8093E80006C08232BA
:1021100009F04DC08F898093070180918306882341
:1021200019F0EEEFFAE002C0E0E0F8E08091000183
:1021300090910101A0910201B0910301803B944074
:10214000A105B10509F07BC08091070180FF93C014
:1021500076C00E94290EDC0112960D911C911397F6
:102160000115110541F1D801ED91FC910190F0812B
:10217000E02DBE016B5E7F4FC8010995811117C02C
:10218000F80100851185ECCF113009F44EC01330F1
:1021900091F48F89882309F445C0823081F440E8A6
:1021A00067E082EF9FE00E947115882321F08EEF97
:1021B0008093E80079C081E28093EB0075C08130A4
:1021C00029F440E86BE086EE9FE0EDCF833099F78D
:1021D0000E94290EDC011296ED90FC9013978E015F
:1021E0000F5F1F4F6801E114F10479F0D701ED9101
:1021F000FC910680F781E02DB801C7010995080F11
:10220000111DF701E084F184EECFD8011C92F60194
:1022100001900020E9F73197BF016C197D0940E07A
:10222000C601C1CF60ED7FE002C064ED7FE06115C3
:10223000710509F2FB01449150E080E840CF0FB6F0
:10224000F894A89580916000886180936000109256
:1022500060000FBEA895EE3F2AE0F20739F08091AA
:10226000FE0A9091FF0A91838083A1CF1092FF0A0A
:102270001092FE0A9CCFEE3F8AE0F80731F0808191
:1022800091819093FF0A8093FE0A87E797E79183F5
:1022900080839BE088E10FB6F894A8958093600056
:1022A0000FBE9093600083CF6C960FB6F894DEBF9C
:1022B0000FBECDBFDF91CF91FF91EF91BF91AF9155
:1022C0009F918F917F916F915F914F913F912F914E
:1022D0001F910F91FF90EF90DF90CF900F900FBE66
:1022E0000F901F901895789484B5826084BD84B552
:1022F000816084BD85B5826085BD85B5816085BD01
:1023000080916E00816080936E00109281008091B8
:102310008100826080938100809181008160809340
:102320008100809180008160809380008091910085
:1023300082608093910080919100816080939100F0
:10234000809190008160809390008091C1008460B2
:102350008093C1008091C10082608093C100809110
:10236000C10081608093C1008091C300816080932F
:10237000C3008091C00082608093C0008091C20041
:1023800081608093C20080917A00846080937A009B
:1023900080917A00826080937A0080917A008160D7
:1023A00080937A0080917A00806880937A001092FE
:1023B000040210928406109202028091D70081607C
:1023C0008093D70080EA8093D80089B5806189BD69
:1023D00089B5826089BD09B400FEFDCF61E070E07F
:1023E00080E090E00E94340A8091D8008F7C806168
:1023F0008093D8008091E000807F8093E0008091FE
:10240000E1008E7E8093E1008DE08093E200559A9A
:10241000209AEEEFFFE7859194918B3F9C4D19F444
:1024200081E08093830681EC80937C0085B1806F8E
:1024300085B9249884B1866E84B95E9A5F988AB112
:10244000806D8AB9769A6E9881B3806F81BB8998C6
:1024500080B38D7080BB80E58CBD81E08DBD85E053
:1024600090E00E949E0C5F9A85E090E00E949E0C96
:102470005E985C98CCE5D1E01C2F135FFE0184913F
:102480000E94B60C21961C13F9CF5C9A81E88093C8
:10249000640081E080936500C0E0D4E080E00E94A9
:1024A000B60C2197D9F70E94A30C87FF1DC085EABF
:1024B0000E94BC0C2E982F982D9880916400806209
:1024C000809364000E94AB0CFDCF2D980E94A30C5A
:1024D0008478843871F00E94A30C8471843131F1C6
:1024E00088EC90E00E949E0C0E94A30C82FDEDCF30
:1024F0003AC00E949C0C88EC90E00E949E0C2F98A1
:1025000082E090E00E940A168F3F29F06FEF82E090
:1025100090E00E94121684EF91E00E949E0C2F9A88
:102520000E94A30C84788438D9F3D5CF0E949C0CE8
:1025300088EC90E00E949E0C2E9882E090E00E9431
:102540000A16882329F060E082E090E00E941216CB
:1025500084EF91E00E949E0C2E9A0E94A30C84713D
:102560008431D9F3BDCF0E949C0C82E090E00E94A0
:102570000A16882319F00E94C60C02C00E94C10CE2
:102580002E98CEEEDFEF08E010E00E94A30C86FF4D
:1025900004C02E9A2F9A2D9A8BC0CC3F2FEFD207D2
:1025A00019F42E9A2F9805C0C831D10511F42F9A2D
:1025B0002D980E940A0EC03F4FEFD40784F40E946A
:1025C000170E8BE190E00E949E0CC03F5FEFD50795
:1025D00009F059C08AEF90E00E949E0C54C09E0101
:1025E000D7FF04C0222733272C1B3D0B277033272E
:1025F000CE01D7FD079673E0959587957A95E1F71B
:10260000D7FF05C00197F801E21BF30B9F017C0186
:10261000F694FE2CEE24F794E79460E070E0380125
:10262000621A730AA70140585F4F5A018F3F5FEF4C
:10263000950744F40196685A7F4F7501603B710518
:1026400089F7BDCFD701A756BD4F40E050E08F3F7F
:10265000EFEF9E0709F4ABC1FA01E60FF71FE4554F
:10266000FF4FE4916D01CA18DB08CE0CDF1CF0E0CF
:102670001F01022E01C0220C0A94EAF7F6015080D5
:102680002528208294C12196C931D10509F07DCF3A
:102690008CEB92E00E949E0C0E949C0CE0910C0638
:1026A000F0910D060190F081E02D8CE096E0099507
:1026B00082E390E00E949E0C0E94A30C8111F8CF4F
:1026C00081E08093240680E18093130685E00E94D8
:1026D000250C8DE00E94250CECE6F1E0E491809160
:1026E0007B00E3FB882480F8912C55E0880C991C32
:1026F0005A95E1F78F7D882A80927B00E770E0642D
:10270000E0937C0080917A00806480937A008091CD
:102710007A0086FDFCCF609178008091790070E0AE
:10272000782B072E000C880B990B6115710581051C
:10273000910511F00E940116C3E4D1E0C12CD12C07
:102740007601CA94F1E0C33CDF07A1F000E010E09D
:102750000E94FC155E01A00EB11EA70196010E9409
:102760002016F50160830F5F1F4F0830110581F7B8
:102770002896E8CFC3ECD1E030ECC32ED12CE12C6D
:10278000F12C21E0C33ED20771F00E94FC15A70195
:1027900096010E942016DC01CB010896A11DB11DF7
:1027A00089939993EECF25E7222E21E0322E2FB781
:1027B000F89480913F0190914001A0914101B09126
:1027C00042012FBF409118065091190660911A06D8
:1027D00070911B0620911C06222341F020911406C3
:1027E000821B80931D0610921C06D9C08417950782
:1027F000A607B70738F4481B423008F4D0C00E943F
:10280000AB0CCDC041E040931C068093140690931E
:102810001506A0931606B093170620911306820F93
:10282000911DA11DB11D8093180690931906A093C8
:102830001A06B0931B0680910F0690911006019620
:102840009093100680930F060E940A0E10922106A4
:102850001092200610921F0610921E0693ECE92E8D
:1028600091E0F92EC0E0D0E08E010D5B1E4F80E4B8
:10287000882E912CA12CB12C2FB7F89460913F0198
:102880007091400180914101909142012FBFF70169
:10289000C080D180D0931F06C0931E0696010D2CD8
:1028A000000C440B550B0E94521624013501420EB8
:1028B000531E641E751EC60160E370E00E948316FD
:1028C0009C01205C3F4F032E000C440B550BC301B1
:1028D000B2010E94521668507109709321066093EC
:1028E00020060E94FC1528EE33E040E050E00E94F4
:1028F00020166A3D73408105910554F00E94FC1535
:102900002FEF30E040E050E00E942016F801608395
:10291000F80161918F01E0910806F091090601909C
:10292000F081E02D88E096E00995F8E08F0E911C8B
:10293000A11CB11C20E882169104A104B10409F085
:102940009BCF289642E0E40EF11CC038D10509F077
:102950008BCF0E94A30C83FF06C087EA0E94BC0CA9
:102960000E94C10C09C00E94A30C82FF05C086EA28
:102970000E94BC0C0E94C60C0E94170E80913E0162
:1029800081110DC030923D0120923C0130923B01FB
:1029900020923A010E94330B51E050933E0180E0B7
:1029A00090E0892B09F403CF0E94000000CF21158D
:1029B000310581F0FA01E60FF71FE455FF4FE4916E
:1029C000F0E0062C02C0F595E7950A94E2F7DC905A
:1029D000ED29EC934F5F5F4F11964835510509F093
:1029E00036CE28CE0F931F93CF93DF938C0181E0D7
:1029F00090E00E940A1680FF31C08AE090E00E94B9
:102A00000A169FEF980F9E3F48F522E330E0D80169
:102A100057963C932E93569728E330E059963C9373
:102A20002E935897CBE0D0E0D801ED91FC91019026
:102A3000F081E02D682FC8010995CE010E940A1689
:102A40002196C131D10581F70E94170E88EE93E0DF
:102A5000DF91CF911F910F910C949E0CDF91CF913C
:102A60001F910F91089504970C94F214E3E3F6E09C
:102A70001382128288EE93E0A0E0B0E08483958315
:102A8000A683B78386E191E0918380838FEF9FEFE8
:102A900095878487E8E0F6E0138212821186128619
:102AA00020E1238790878783108A118A128A138AEC
:102AB000148A86E291E09183808380E391E095839C
:102AC0008483178A168A118E108E81E0828F138E6E
:102AD000848F158E80E299E0909306068093050618
:102AE0000895CF92DF92EF92FF920F931F93CF93AF
:102AF000DF931F92CDB7DEB7182F062FE42E862F57
:102B0000880F8E5F99830E94AF0E83E00E94AF0E04
:102B1000F12EC12E9981D92E8C2D8F19801798F402
:102B2000F601E7FE02C0849101C080810E94AF0ED1
:102B3000182F80E00E94AF0E8123FFEFCF1ADF0A2B
:102B40008111EACF01C081E00F90DF91CF911F91F9
:102B50000F91FF90EF90DF90CF9008958F929F920A
:102B6000AF92BF92CF92DF92EF92FF92CF93DF931B
:102B7000EC01688179818A819B81611571058105EC
:102B8000910521F464E279ED8BE597E02DE133EFD7
:102B900041E050E00E94201649015A019B01AC011E
:102BA000A7EAB1E40E943F166B017C01ACEEB4EFE2
:102BB000A50194010E944D16DC01CB018C0D9D1DD9
:102BC000AE1DBF1DB7FF03C00197A109B0488883A0
:102BD0009983AA83BB83BC01CD019F77DF91CF91FD
:102BE000FF90EF90DF90CF90BF90AF909F908F902D
:102BF00008950E94AE1508958CE091E00E94AE15F4
:102C0000089560930C0170930D0180930E019093D1
:102C10000F010895F999FECF92BD81BDF89A9927C9
:102C200080B50895262FF999FECF1FBA92BD81BDB8
:102C300020BD0FB6F894FA9AF99A0FBE019608953E
:102C4000052E97FB1EF400940E94371657FD07D0FF
:102C50000E94521607FC03D04EF40C943716509580
:102C60004095309521953F4F4F4F5F4F0895909578
:102C70008095709561957F4F8F4F9F4F08950E946B
:102C80007416A59F900DB49F900DA49F800D911D6B
:102C900011240895B7FF0C943F160E943F16821B23
:102CA000930B0895A1E21A2EAA1BBB1BFD010DC0B8
:102CB000AA1FBB1FEE1FFF1FA217B307E407F507EC
:102CC00020F0A21BB30BE40BF50B661F771F881FC8
:102CD000991F1A9469F760957095809590959B015E
:102CE000AC01BD01CF010895A29FB001B39FC00107
:102CF000A39F700D811D1124911DB29F700D811D28
:102D00001124911D089597FB072E16F4009407D007
:102D100077FD09D00E94971607FC05D03EF49095E8
:102D200081959F4F0895709561957F4F0895AA1BD7
:102D3000BB1B51E107C0AA1FBB1FA617B70710F0A6
:102D4000A61BB70B881F991F5A95A9F780959095D8
:102D5000BC01CD010895EE0FFF1F0590F491E02D09
:102D6000099481E090E0F8940C94B616F894FFCFA3
:102D700000E1000000000000FFFFFFFF0100000075
:102D8000030100000000F60C730D590D170D350DF1
:102D90000C0D0000000023092808F214FCFF0000BD
:0A2DA000331500C18081000000001F
:2070000055C000006EC000006CC000006AC0000068C0000066C0000064C0000062C0000043
:2070200060C000005EC00000F2C400005AC0000058C0000056C0000054C0000052C00000EE
:2070400050C0000078C000004CC000004AC0000048C0000046C0000044C0000042C00000BE
:2070600040C000003EC000003CC000003AC0000038C0000036C0000034C0000032C0000048
:2070800030C000002EC000002CC000002AC0000028C0000026C0000024C0000022C00000A8
:2070A00020C000001EC000001CC0000011241FBECFEFDAE0DEBFCDBF11E0A0E0B1E0E2E3BC
:2070C000FFE702C005900D92A83AB107D9F711E0A8EAB1E001C01D92AE3BB107E1F78FD30B
:2070E00026C78ECFF89410926F0010928100109285001092840081E085BF15BE47985D9AEB
:20710000289A0C94000008952091B2013091B3012F5F3F4F3093B3012093B201932F37FFA6
:2071200003C08EEF831B982F990F921710F447980895479A08951F920F920FB60F9211246E
:207140002F938F939F93EF93FF9310928500109284008091A8019091A901009741F00197D3
:207160009093A9018093A801892B09F45D9A8091AA019091AB01009741F001979093AB0126
:207180008093AA01892B09F4289AE0E0F0E0859194918F5F9F4F49F08091AC019091AD0151
:2071A00001969093AD018093AC01FF91EF919F918F912F910F900FBE0F901F90189584E0BC
:2071C0008093E9000DC08091E8008B778093E80003C08EB3882351F08091E80082FFF9CFBE
:2071E0008091E80085FFEFCF8091F1000895982F83E08093E9008091E80085FD0DC0809136
:20720000E8008E778093E80003C08EB3882369F08091E80080FFF9CF9093F1005D9884E6CB
:2072200090E09093A9018093A80108954F925F926F927F928F929F92AF92BF92CF92DF921E
:20724000EF92FF920F931F93CF93DF9384E08093E9008091E80082FF57C2289884E690E067
:207260009093AB018093AA01AADF182F853481F48CE49DE19093AD018093AC0107B600FC4B
:20728000FDCFF999FECF81E180935700E89503C0843519F494DF8DE00DC28C34E1F38035F9
:2072A000D1F3843721F484E4A2DF80E003C2813611F489E5FFC18134B1F481DF182F7FDFE3
:2072C00090E0880F991FAA2797FDA095BA2F312F330F20E0442737FD4095542F822B932B68
:2072E000A42BB52BB8C1803711F483E5E3C1833549F4C0E0D1E089917ADF21E0C730D20714
:20730000D1F7D9C1863521F481E371DF80E3D2C1833731F487E86BDF85E969DF8EE1CAC149
:207320008536B9F4E0E0F0E093E085E090935700E89507B600FCFDCF80935700E89507B65D
:2073400000FCFDCFE058FF4FA0E7E030FA0771F7A2CF823739F4E1E0F0E089E08093570024
:207360008491A8C1863439F4E0E0F0E089E08093570084919FC18E3439F4E3E0F0E089E0E5
:2073800080935700849196C1813539F4E2E0F0E089E08093570084918DC1823631F489E521
:2073A00026DF80E024DF80E885C1823419F0873609F0E5C01092AD011092AC0100DF082FE8
:2073C000FEDEF82EFCDE682E8554823008F071C1902F80E0CF2DD0E0C82BD92B10926F00B3
:2073E000173609F04BC081E180935700E895DD24CC24C3943FC0E090AE01F090AF010091CC
:20740000B0011091B101B6E46B16D9F4ED2DF0E0EE29FF29E4918E2FEADEDD2081F082E08D
:2074200090E0A0E0B0E0E80EF91E0A1F1B1FE092AE01F092AF010093B0011093B101DC2470
:2074400018C0D801C701B695A7959795879559D5CEDE82E090E0A0E0B0E0E80EF91E0A1FF2
:207460001B1FE092AE01F092AF010093B0011093B1012197209709F0BECF7DC08090AE01F5
:207480009090AF01A090B001B090B10196E4691609F05DC083E0F40180935700E89507B63E
:2074A00000FCFDCF54C0F6E46F1661F5772031F1E090AE01F090AF010091B0011091B1019E
:2074C0007EDED82ECC24852D90E08C299D29F7010C0140925700E895112482E090E0A0E08B
:2074E000B0E0E80EF91E0A1F1B1FE092AE01F092AF010093B0011093B10102C060DE582E1A
:20750000742423C0E090AE01F090AF010091B0011091B10116950795F794E79450DE682FFA
:20752000C701F7D48091AE019091AF01A091B001B091B1010296A11DB11D8093AE01909349
:20754000AF01A093B001B093B101219704C05524772444244394209709F0A5CF96E46916B6
:2075600041F485E0F40180935700E89507B600FCFDCF8DE03CDE82E080936F009CC0833492
:2075800071F40091AE011091AF0119DE90E021E0F8010C0120935700E89511247CCE8336C8
:2075A00019F5E090AE01F090AF010091B0011091B10105DEF701E16090E021E00C0120938C
:2075C0005700E895112482E090E0A0E0B0E0E80EF91E0A1F1B1FE092AE01F092AF0100936A
:2075E000B0011093B10157CE8D3661F4E091AE01F091AF0185E080935700E89507B600FCF2
:20760000FDCF49CE823551F4E091AE01F091AF0105911491812FEBDD802F4CC0843421F5FE
:20762000E090AE01F090AF010091B0011091B10116950795F794E794C2DD682FC70169D4DE
:207640008091AE019091AF01A091B001B091B1010296A11DB11D8093AE019093AF01A093D8
:20766000B001B093B10117CE843609F5E090AE01F090AF010091B0011091B101D801C70142
:20768000B695A795979587953CD4B1DD82E090E0A0E0B0E0E80EF91E0A1F1B1FE092AE010A
:2076A000F092AF010093B0011093B10104C08B3111F08FE39CDD83E08093E9009091E8002B
:2076C0008091E8008E778093E80095FF04C010C08EB38823C9F08091E80080FFF9CF809193
:2076E000E8008E778093E80003C08EB3882361F08091E80080FFF9CF84E08093E9008091F1
:20770000E8008B778093E800DF91CF911F910F91FF90EF90DF90CF90BF90AF909F908F90AC
:207720007F906F905F904F9008959091B601892F8F77813249F58091B7018032A1F081328A
:2077400019F5913A09F58091E800877F8093E8008DE091E067E070E00BD28091E8008B770B
:207760008093E8000895913279F48091E800877F8093E8008DE091E067E070E05DD2809192
:20778000E8008E778093E800089582E061EC42E0B5D083E061E842E1B1D084E060E842E1EF
:2077A000ADC084B7877F84BF88E10FB6F89480936000109260000FBE20E880E090E00FB63F
:2077C000F89420936100809361000FBE81E085BF92E095BF3F9A209A559AE1E6F0E02083A1
:2077E000108247985D9A289A109289008AEF8093880090936F0083E080938100F0C0409116
:20780000000850910108109201081092000894B714BE88E10FB6F8948093600010926000D5
:207820000FBE292F30E0F901E270F07091FD18C090FF05C0859194918F5F9F4F81F423FFFF
:207840000FC08091090190910A014817590741F0E0E0F0E0859194918F5F9F4F09F042DC64
:20786000A0DF78941092AD011092AC010CC0DEDC36D38091AC019091AD0181549F4110F00D
:207880001092140141DC80911401882381F78091E00081608093E00025DC80E090E0089598
:2078A000FA01923049F0933061F09130F9F485E191E022E130E01EC087E291E02EE330E04D
:2078C00019C0882329F485E691E024E030E012C0813029F489E691E022E230E00BC0823006
:2078E00029F48DE891E028E130E004C080E090E020E030E091838083C90108958093E9004E
:207900008091EB0081608093EB001092ED006093EC004093ED008091EE00881F8827881F62
:2079200008958091B60188238CF403C08EB38823B1F08091E80082FFF9CF8091E8008B772A
:207940008093E80008958EB3882349F08091E80080FFF9CF8091E8008E778093E800089594
:20796000EF92FF920F931F9345D04CD008ED10E0F80180818F77808380818068808380819B
:207980008F7D808319BC1EBA1092B40180EEE82EF12CF70180818B7F8083F8018081816052
:2079A000808380E060E042E0A9DFE1EEF0E080818E7F8083E2EEF0E0808181608083808144
:2079C00088608083F70180818E7F8083F8018081806180831F910F91FF90EF900895E7ED06
:2079E000F0E08081816080838AE482BF81E08093B501B6CFE8EDF0E080818E7F808310921C
:207A0000E20008951092DA001092E10008951F920F920FB60F9211242F933F934F935F93F6
:207A20006F937F938F939F93AF93BF93EF93FF938091DA0080FF1BC08091D80080FF17C0B2
:207A40008091DA008E7F8093DA008091D90080FF0BC080E189BD82E189BD09B400FEFDCF36
:207A600081E08EBB3BD203C019BC1EBA37D28091E10080FF17C08091E20080FF13C0809138
:207A8000E2008E7F8093E2008091E20080618093E2008091D80080628093D80019BC85E049
:207AA0008EBB1CD28091E10084FF2CC08091E20084FF28C080E189BD82E189BD09B400FEC5
:207AC000FDCF8091D8008F7D8093D8008091E1008F7E8093E1008091E2008F7E8093E20012
:207AE0008091E20081608093E2008091B401882331F48091E30087FD02C081E001C084E067
:207B00008EBBECD18091E10083FF21C08091E20083FF1DC08091E100877F8093E10082E06A
:207B20008EBB1092B4018091E1008E7F8093E1008091E2008E7F8093E2008091E2008061E9
:207B40008093E20080E060E042E0D8DEC7D1FF91EF91BF91AF919F918F917F916F915F9130
:207B60004F913F912F910F900FBE0F901F9018959C014091BC015091BD014617570718F49D
:207B8000F90190E044C06115710511F0AB01F8CF8091E8008E778093E80040E050E0F0CF0F
:207BA0008EB3882309F444C0853009F443C08091E80083FF02C081E008958091E80082FD70
:207BC00031C08091E80080FF22C08091F3009091F200782F60E0292F30E0262B372B07C07A
:207BE00081918093F100415050402F5F3F4F4115510519F02830310598F390E02830310566
:207C000009F491E08091E8008E778093E8004115510531F6992321F605C08EB3882341F075
:207C2000853041F08091E80082FFF7CF80E0089582E0089583E008959C016115710529F47C
:207C40008091E8008B778093E800F90126C08EB3882391F1853091F18091E80083FF02C06C
:207C600081E008958091E80082FFF1CF06C08091F10081936150704059F02091F300809191
:207C8000F200322F20E090E0822B932B892B79F78091E8008B778093E80061157105B9F601
:207CA00005C08EB3882341F0853041F08091E80080FFF7CF80E0089582E0089583E00895C2
:207CC0000F931F93DF93CF9300D0CDB7DEB7E6EBF1E08091F100819381E0EE3BF807C9F792
:207CE00024DD8091E80083FFE4C08091B6019091B701953009F46DC0963040F4913081F1A7
:207D0000913070F0933009F0D4C02AC0983009F4A3C0993009F4B2C0963009F0CAC07CC023
:207D2000803809F4C6C0823809F0C3C08091BA0187708093E9008091EB001092E9002091DB
:207D4000E800277F2093E80090E025E0969587952A95E1F781708093F1001092F10087C0D8
:207D6000882319F0823009F0A4C08F71823009F0A0C08091B801882331F52091BA01277097
:207D800009F497C02093E9008091EB0080FF1BC0933021F48091EB00806213C08091EB0018
:207DA00080618093EB0081E090E002C0880F991F2A95E2F78093EA001092EA008091EB00E5
:207DC00088608093EB001092E9008091E800877F51C0882309F06DC01091B8011F770FB79B
:207DE000F8948091E800877F8093E8009ADD8091E80080FFFCCF8091E3008078812B809398
:207E0000E30080688093E300112311F482E001C083E08EBB0FBF4DC08058823008F049C033
:207E20008091B8019091B9016091BA01AE014F5F5F4F36DDBC01009709F43BC08091E8008E
:207E4000877F8093E80089819A8192DE8091E8008B778093E8002DC0803859F58091E800AA
:207E6000877F8093E8008091B4018093F1008091E8008E778093E80054DD1BC08823C9F4CA
:207E80009091B8019230A8F48091E800877F8093E8009093B40145DD8091B401882331F420
:207EA0008091E30087FD02C081E001C084E08EBB6CDC8091E80083FF0AC08091EB0080624E
:207EC0008093EB008091E800877F8093E8000F900F90CF91DF911F910F91089508951F9360
:207EE0008EB3882361F01091E9001092E9008091E80083FF01C0E4DE17701093E9001F916F
:207F00000895F999FECF92BD81BDF89A992780B50895262FF999FECF1FBA92BD81BD20BDBD
:207F20000FB6F894FA9AF99A0FBE01960895F894FFCF4341544552494E4100777700080031
:207F40000000000000080112011001020000084123360001000201000109023E00020100FF
:207F600080320904000001020201000524001001042402040524060001070582030800FF0C
:207F800009040100020A000000070504021000010705830210000104030904220341007216
:207FA000006400750069006E006F0020004C0065006F006E006100720064006F0000001836
:1A7FC00003410072006400750069006E006F0020004C004C004300000000D7
:00000001FF
